:020000040000FA
:100000002500000C02000C0C060006058604A60460
:100010005E0946070F0A6607130A5509060A5509BD
:100020006607060A170A55094607060A170A8605CB
:100030005E095E095E094607200A6607200A060A6D
:100040005E095E0986050D0C28003C09100C28008D
:100050003C09000C28003C090D0C28003C09A605B1
:100060005E095E095E095E095E095E095E095E0958
:100070005E095E09A604060A090C29000604450962
:10008000E9024E0A060545090008870C2A00EA0223
:10009000470A870C2A00EA024B0A000828030307D4
:1000A000530A06053F0A06043F0AC50C2900000052
:1000B000000000000000E9025A0A0008C80C2B00EA
:1000C0005509EB02600A400C2900E902650A0008A4
:021FFE00EA0FE8
:00000001FF
